:020000040800F2
:10500000581A0020D5500008B9820008DD7A00083F
:105010000000000000000000000000000000000090
:105020000000000000000000000000006590000883
:10503000000000000000000041890008799100088C
:10504000E7500008E7500008E7500008E750000864
:10505000E7500008295B0008E7500008E750000807
:1050600000000000E7500008515A0008E75000080F
:10507000E7500008357F000800000000E7500008F6
:1050800000000000E75000080000000000000000E1
:10509000E750000800000000E7500008E750000853
:1050A000E7500008E7500008E75000080999000899
:1050B000E7500008E7500008000000000000000072
:1050C0000348854600F060FC004800471DA7000823
:1050D000581A00200448804704480047FEE7FEE7CE
:1050E000FEE7FEE7FEE7FEE715920008C150000864
:1050F00030B50B46014600202022012409E00D4670
:10510000D5409D4205D31D469540491B25469540F7
:1051100040191546521E002DF1DC30BDF0B51FB40C
:105120000646002082B005464024019100901BE015
:10513000019922460F46304600F04EFB049A059B2B
:10514000801A994110D310461946224600F034FBCC
:10515000361A8F410197224601200021009F00F05E
:105160002BFB38184D4100902046641E0028DFDCE0
:10517000019B00982946324607B0F0BD03460B4319
:105180009B0703D009E008C9121F08C0042AFAD2FD
:1051900003E00B780370401C491C521EF9D2704783
:1051A000D2B201E00270401C491EFBD270470022BF
:1051B000F6E710B513460A4604461946FFF7F0FF16
:1051C000204610BD30B504460020034600E05B1CBD
:1051D000934203D2E05CCD5C401BF8D030BDF8B503
:1051E00002464A40D40F42004B0052085B089A42E4
:1051F00002D20246084611464A0023D0C30D4A0097
:10520000DDB2120EAD1A202D35DA49020126490A07
:10521000F6058A19002C00D0524220214F1B11465E
:10522000B9402A411018C20D9A4221D0002C17D043
:10523000012D08DCDA05801AD20F8019D207DBB203
:1052400000F0F6FAF8BDDA05801A012340001B06CB
:10525000C01880185A428018CA0F1043490007E04E
:105260004908C2071143DA05801A801940088018DE
:1052700000F0D6FAF8BD61000122511A001BF7E7D1
:105280000122D2075140AAE70122D2075040A6E7E7
:1052900070B502464A40D50F40004A00ED0740086D
:1052A0005208002814D0002A12D0C40DD30D410298
:1052B0000120C0055202490A520AE41A09181218BC
:1052C0007D34914201D3641C00E04900002C01DAD6
:1052D000002070BD0023914201D3891A0343400886
:1052E00049000028F7D100290AD0914202D10121BA
:1052F000C90705E0914201D2012101E00121C94322
:10530000E005C018401900F08BFA70BDF0B50746F3
:105310000846584087B0C00F049048000E46590018
:1053200040084908BC1A884105D2384631461E4615
:1053300017460B4602465800400810434CD0300D2B
:10534000039040055900400D490D0590401A029008
:10535000402872DA18030121000B09050843019067
:1053600004980092002805D00199524200208841FB
:1053700000920190029840210A1A0199009800F0C9
:105380001BFA05460C466B4607CB00F036FAC019EF
:105390007141039A0E0D0023D71756401A467A40E2
:1053A000164344D0049A002A2DD0029A012A039A67
:1053B00015DC1205C01A914101263605001C714109
:1053C000D20F059ED2070093019202962A462346E9
:1053D00000F074FA07B0F0BD38463146FAE716051A
:1053E000224A0F46B218C01AB74101210905001C14
:1053F0004F4100187F41114618187941E20F1043C0
:105400006D19644113E0E2076D0815436408C20793
:105410001443039A01261205C01A91413605001C57
:105420007141CE07400830434908C01851412A460F
:10543000234600F036FACDE7FFE70498012240004A
:10544000C117121A00238B4104983146C417381A29
:10545000A141EEE730B40124E407634030BC55E7D6
:1054600030B40124E407614030BC4FE70000E0FFA6
:10547000F0B51FB488B00B990998002448400999E9
:10548000C00F490049080991C0070B9900904900D5
:1054900049080B9109990898A64608431CD00B9916
:1054A0000A98084318D0099801244000420D48008A
:1054B000410D099824050003000B204309900B9827
:1054C0000003000B20430B9050181C494018002289
:1054D00001901446104605E0002001460DB0F0BDD5
:1054E000032801DA034600E003239C46C11A0AAEF2
:1054F0000AE05F0008ADED5B4F00F75B7D430027DE
:10550000AA187C41491C5B1E6145F2DD410004ABD9
:105510005A522104120C0A43240C401C0828DFDBD9
:10552000019802900099704601910090059B049AA1
:105530000799069800F0C2F9D0E700000DFCFFFFC4
:10554000F0B50C465C4085B0E40FE40703944C00D2
:1055500000266408590094464908024602962243F0
:1055600021D062460A431ED06200570D4A000E0346
:105570002303550D012402462C492405781B1B0BDF
:10558000360B401823432643614600901C46501AB0
:10559000B44103D30098401C009002E09218009898
:1055A0005B41002803DA0020014605B0F0BD002071
:1055B000012109050746864611E064461D46141B75
:1055C000B54106D36546521BB341744607430C43AD
:1055D000A646CD0740084908284392185B41054676
:1055E0000D43EAD11046184313D060461946504087
:1055F0007140084306D06046101AB34106D201221A
:10560000002306E000220123DB0702E00122D2434F
:105610005310009874460105381C6141029C039D9B
:105620000019694100F03DF9BFE70000FD030000EB
:10563000C217C10F504010B54018CA079623002169
:1056400000F0F6F810BD10B500229623114600F0C8
:10565000EFF810BD0EB5C217C10F5040CA07401871
:105660000021054B0293019200910A460B4600F07F
:1056700025F903B000BD0000330400000EB5054954
:105680000291002100910A460B46019100F016F9A3
:1056900003B000BD33040000410040020122400A73
:1056A000D205090E80187F2901DA0020704796295B
:1056B00003DC9622511AC8407047963988407047DB
:1056C00070B5CD0F4A0009030123090B1B051943CF
:1056D0000B4BED070024520D9A4201DA002070BDF9
:1056E000074B34339A4203DC9A1A00F075F802E053
:1056F0000449511888402C43F1D0404270BD00004D
:10570000FF030000CDFBFFFF4A0009030123090B43
:105710001B051943094B10B5520D9A4201DA0020BE
:1057200010BD064B34339A4203DC9A1A00F054F849
:1057300010BD03495118884010BD0000FF03000050
:10574000CDFBFFFFC20FD207400040080BD0C10DB8
:105750000723DB01C91840020905400A1143C208AA
:10576000400711437047002001467047CB0FDB070D
:10577000490010B5490802460A4307D00A0D07241C
:105780000903E401090B121B002A01DC002010BDF3
:10579000C900440F0C43C100E018D205801800F086
:1057A0003FF810BD0122D207002800DB101A0029A3
:1057B00000DB511A8142704710B5202A04DB0146F4
:1057C000203A9140002010BD914020239C1A0346AE
:1057D000E3401943904010BD10B5202A04DB084671
:1057E000203AD040002110BD0B46D340D0402024A9
:1057F000A21A91400843194610BD10B5202A06DBB5
:10580000CB170846203A1041C1170B4306E00B4660
:105810001341D0402024A21A91400843194610BDDC
:10582000002904DA401C490001D1400840007047BB
:1058300070B40024050C05D11024000402D1002905
:1058400021D01124050E01D100020834050F01D129
:105850000001241D850F01D18000A41C002801DB5C
:105860004000641C002908D020252E1B0D46F54061
:10587000A14000D001212943084301061B1B000A57
:10588000DB1D02D5002070BC7047DB05181880189E
:105890000029F8DA401C4900F5D170BC40084000EE
:1058A000704710B5002B08DA0024401C61419218A3
:1058B0005B411A4301D14008400010BDF0B51FB450
:1058C00082B005460C0003D0084604F0DDF802E083
:1058D00004F0DAF820300246009021462846FFF70F
:1058E0006BFF049B059A04460F4618431143084377
:1058F00014D0184610431BD0009840210A1A1846AD
:105900000599FFF769FF05460E46009A0599049828
:10591000FFF752FF084305D0012004E02046394636
:1059200007B0F0BD0020C11705430E432C43374399
:1059300000990E986305401A7905E40A00220C4389
:10594000FD0A0A3002D500200146E9E701051019D9
:1059500069410C9C0D9D00196941FFF7A2FFDFE72B
:1059600010B5002904DB0124E40740428C412146A4
:10597000002B04DB1C460123DB075242A341994262
:1059800000D1904210BD0000064C0125064E05E0F6
:10599000E36807CC2B430C3C98471034B442F7D350
:1059A000FFF792FB8CAA0008ACAA000838B50446A1
:1059B000064805490068FFF79BFB604300E0401E76
:1059C00000900028FBD138BD40420F000C010020A0
:1059D000F8B50446006881688907890F012902D15A
:1059E0000168C90722D18168114A1026114001259A
:1059F00000290ED18168294381600120FFF7D6FF7D
:105A000000F0BCFF07460CE000F0B8FFC01B0A28FE
:105A100007D9606D30436065A06D2843A065012003
:105A2000F8BD20680068C043C007EDD10020F8BD74
:105A30001700008010B500231A4603E0845CE318C9
:105A40009BB2521C8A42F9D3D84380B210BD0000E9
:105A500010B5034800F052FD024800F04FFD10BDA4
:105A6000F8150020B015002030B5446C1C252C40E2
:105A70000125A540046C6560046863608368102B91
:105A8000036803D099600068C26030BD9A60006806
:105A9000C16030BD1449012048720A4602205E32BE
:105AA000507203203C3A507204200E3A50720F4854
:105AB0000D4B0078087022310870203108770C49AE
:105AC0005A1C0878587149789971233318715971A3
:105AD000203318775977107551751A461E32107594
:105AE000517510765176704740110020C700002094
:105AF000E400002010B503F08DFA202003F032FB03
:105B0000012004F071FB002003F02CFB044804F09A
:105B10000FFA044804F0B2FC002004F0E7FC10BDCA
:105B2000B00000208380000070B50520012100072F
:105B300000F014FF0025154C002800D06560144EBD
:105B40000221304600F00AFF002817D10120207002
:105B50007F20C005A0600F48808F002805D001215C
:105B600000228902304600F002FF0B486560008881
:105B70000A2148430949088003F0D8FE012000F0BB
:105B800025FE022000F022FE70BD0000FC00002077
:105B900000040050400D0020D4000020E000002050
:105BA0007047000010B5084900224A6107494B6858
:105BB0004C1523434B604B68082423434B60C009BA
:105BC000C001026010BD000040160020002002400D
:105BD0007FB500250C460646039500F0C7FDE00999
:105BE000029003A901960095684600F057FD002831
:105BF00004D000F08FFD002004B070BD00F08AFDDD
:105C00000120F9E710B5002302E0C45CCC545B1C12
:105C10009342FAD310BD000010B5214A00219069CB
:105C2000C305204804D541690223194341619115F8
:105C300093699B0505D543690124234343616302AE
:105C4000194393695B0505D54369082423434361E0
:105C5000E301194393691B0505D5436904242343D4
:105C600043616302194393699B0405D5436910247A
:105C7000234343616302194393699B0304D5446939
:105C800020231C43446119439369DB0305D5436911
:105C9000402423434361A0020143916110BD0000F1
:105CA000002002404016002070B5054600F066FE58
:105CB0000646184C0AE0681C08D0002D04D000F0FD
:105CC0005DFE801BA84201D9032070BDA069C007FA
:105CD000F1D1A069800701D50220A061A069C005AB
:105CE00011D4A06980050ED4A06940050BD4A06929
:105CF000000508D4A069800405D4A069800302D4FB
:105D0000A069C00303D5FFF787FF012070BD002005
:105D100070BD000000200240F8B517460026054679
:105D20000C4600F023FD09E029460220226800F01D
:105D3000FFFC002804D1241D2D1D361DBE42F3D3C7
:105D400000F0E8FCBE4201D20020F8BD0120F8BD01
:105D500010B5084902460020054B497905E044008A
:105D60001C5B944203D0401CC0B28842F7D310BDE4
:105D7000681200204800002010B500F0F4FD10BDAE
:105D800010B5094800F0BCFF80B2FFF777FC074A66
:105D9000074BFFF76DFB0022064BFFF7D1FBFFF728
:105DA000B3FC80B210BD0000A8140020F853E3A596
:105DB0009B843E4000408F40F8B540493E488A7F72
:105DC0000275C97F41753E490A7802764978417665
:105DD00039490520133148720A2004F03FFB7D2029
:105DE000C00004F055FB3449002213310C2004F0AC
:105DF0001FFC00210C2004F02DFC022004F07EFB8F
:105E0000304D2E4C00210F2004F0A8FA28422063C8
:105E1000F8D0206B411C40D02B4E2C4F40043ED577
:105E20008122D20100210F2004F0D7FB0021102095
:105E300004F094FA41062048490E0022633004F031
:105E4000C3FA1D4D6335687A052825D102221C4905
:105E5000681DFFF7B7F900281ED1A87C60711748AC
:105E60000422691C4430FFF789F9606C00F034F8B3
:105E7000A083607929464200133108465130FFF76C
:105E80007DF9134831888088FFF732F9388841431B
:105E90001048018003202070F8BD02F031FAA08B79
:105EA00031880546FFF724F93888414309486D1EBB
:105EB0000180A583F8BD0000A1110020480000204A
:105EC000E400002000D02724D0000020CE000020D5
:105ED000400D0020CC00002010B504460E4800F014
:105EE0000FFF0E49C006C00E098805E02246C240D9
:105EF000D2070FD0401CC0B28842F7D3012005E082
:105F00002246C240D20705D0401CC0B28842F7D317
:105F1000491EC8B210BD0000A8140020D000002007
:105F200010B5084800F096FA0A21064800F032FA47
:105F3000044800F01DF9800503D5024800F01AF965
:105F400080B210BD4C140020F8B52F4D0022012165
:105F5000284600F00CFDFFF7E3FFFFF774FB2B4E24
:105F60003146FFF795F92A4C0122A06011462846D8
:105F700000F0FDFC2749A068002588423EDB207820
:105F8000254F002815D02570FFF7CAFFFFF75BFBF0
:105F90003146FFF77DF9A060FFF7D4FB00223B46B6
:105FA000FFF758FA00221D4BFFF762FAFFF7DEFBFE
:105FB0006060A068FFF7C6FB00223B46FFF74AFA85
:105FC000174A184BFFF754FA06460F466068FFF76A
:105FD000B9FB134A144B5242FFF74AFA32463B468A
:105FE000FFF794F9FFF7C2FB10496060884201DDBA
:105FF000616004E0FF21C905C84200D365606068A4
:10600000FFF74AFBC0B2F8BD0004005000401B443B
:10601000240000200000604000000C4000E06440CC
:106020003333333333B33040CCCCEC3F0000C84281
:10603000F8B5054604464035287C0026012808D0DE
:1060400001202874206881688907890F01290ED1F1
:1060500001E00220F8BD0168C90708D0606D202169
:10606000084360650126002028743046F8BD616D44
:10607000FF2201329143022211436165C168890701
:10608000890F0091C16889088900C1602068816812
:1060900092071143816000F071FC07460EE000F0AA
:1060A0006DFCC01B0A2809D9606D022188431021AC
:1060B00008436065002028740120F8BD20688068CE
:1060C0000028ECDB2068C168009A1143C160606D54
:1060D00080088000401C6065C5E70000F8B50646F2
:1060E0000D464036317C01290DD001213174016803
:1060F0008A68520709D5416D20221143416500206D
:1061000030740120F8BD0220F8BD174B6A68D8052D
:1061100047109A42154C8A6A2B6812D05B035B0BBE
:106120001A438A622968490305D5A1680143A16021
:106130000A20FFF73BFC2868800312D5A06838438B
:106140000EE05B035B0B9A438A622968490302D520
:10615000A1688143A1602868800302D5A068B84384
:10616000A06000203074F8BD01100000002701403D
:10617000406D70470068006C7047000070B5040007
:1061800006D0606D264600254036002802D006E085
:10619000012070BDA5653574204600F0D3F8606D10
:1061A000C00603D421688868400705D5606D1021BA
:1061B000084360653574EBE7606DFF220132904360
:1061C00002221043606588688207920F5B48012AAB
:1061D00002D10A68D2072BD1032362689B079A4237
:1061E00005D05B429A4202D05B009A4209D10A690B
:1061F000920092080A6121680A6963681A430A6179
:106200000CE00A69920092080A6181680F229204E8
:106210009143816081686268114381602168CA6826
:1062200018239A43CA602168CA68A3681A43CA60DF
:10623000816801225206914381608168A28E5206D4
:106240001143816020688168C90004D481680122FB
:106250001207114381602068C168394A1140C1604A
:106260002069E168022825D0002001432046203023
:106270000278037B52035B001A431143226B1143E4
:10628000A26992031143E269D20311432268D368E1
:106290001943D160616A0A46FF3AC23A05D0A26A40
:1062A00011432268D3681943D16042780121012A41
:1062B00002D00BE00420D8E70078002823D0606DDE
:1062C000202210436065A06D0843A065E06B0128A3
:1062D00020681FD00169C90703D001694908490036
:1062E000016120684169C908C900416120684169AC
:1062F000A26B11434161A565606D80088000401C60
:106300006065002070BD2068C26801231B041A4329
:10631000C260DBE70269FF239B009A4302612068A9
:106320000269236CA66C1A43636C33431A430261FF
:10633000206802690A430261D3E700000027014098
:106340001902FEFF10B586B0044614216846FEF718
:106350002EFF0E492068884216D10D48416B421528
:1063600011434163C16A01221143C162C06A694697
:106370001040059002200090032001900020029020
:106380000520000700F02EFA06B010BD00240140E1
:1063900000100240F8B504464069254640350E46D7
:1063A00008280BD02068C068C00709D0606D202184
:1063B00008436065002028740120F8BD082700E02C
:1063C0000C2700F0DBFA009011E0701C0FD0002EBB
:1063D00005D000F0D3FA0099401AB04207D9606D99
:1063E000042108436065002028740320F8BD20685C
:1063F00000683842E9D0606D0121490208436065B8
:106400002068C16809058A0F0C21002A1BD12022AF
:10641000125D002A17D10268120714D5826853074B
:106420000122002B08DB43688B434360606D13023D
:1064300098431043606506E0606D20231843606553
:10644000A06D1043A065A069002801D120680160FB
:106450000020F8BD70B5044621680020896849070E
:1064600021D425464035297C01291CD001212974DD
:10647000E169012904D02046FFF7AAFA002811D1CA
:10648000616D0A4A1140FF2201321143616500210A
:10649000A165297422681C21116021688A6804237F
:1064A0001A438A6070BD022070BD0000FEF1FFFF3C
:1064B00070B50024014620314A79022A03D0042114
:1064C000C163012418E0026813680E25AB43136012
:1064D000026813685B085B001360436C1C22134066
:1064E000012215469D40036C5D604A7100220A71CD
:1064F000816B002900D08847204670BDF0B4016C44
:106500000D6801680C68466C1C2304221E40174667
:10651000B7402F420ED067070CD50C68A40602D4F2
:106520000C6894430C60416C19408A40016C4A60CD
:10653000016B1AE00227B74002462F402032002F9D
:1065400017D0A70715D50C68A40605D40C680A2532
:10655000AC430C6001215171446C02211C40036C5E
:10656000A140596000211171C16A002918D0F0BC06
:1065700008470827B7402F4212D0240710D50C68CF
:106580000E25AC430C60446C01211C400B46A3401B
:10659000046C6360C163517100211171416BE4E7C8
:1065A000F0BC704770B504003CD01F48256814212A
:1065B0002818FEF79DFD800060641C4820640221BD
:1065C000204620300246417129681948E36801409D
:1065D000A06866691843236933431843A3691843C5
:1065E000E3691843236A1843084328600121A0681F
:1065F0008903884210D00D488030836A656C1C2165
:106600000D400F26AE40B3438362656C63680D4056
:10661000816AAB400B4383620020E063012151712A
:10662000107170BD012070BDF8FFFDBF0000024079
:106630000F80FFFFF8B504468C4620300179002515
:10664000012909D00126067141790027012905D0C9
:10665000077102252846F8BD0220F8BD02214171CC
:10666000E7632068016849084900016061462046E7
:10667000FFF7FAF9206B00282068016801D00E228C
:1066800005E0042291430160206801680A22114359
:1066900001602068016831430160DBE7F8B51A4EFC
:1066A0000546307C0F46012807D00120307417487A
:1066B000FFF7FAFA010002D021E00220F8BD002025
:1066C000C04338606C6814E02046FFF76BFA0F484F
:1066D000FFF7EAFA01460E48426808239A434260EF
:1066E000426843159A434260002901D03C6006E0AD
:1066F0008034A8686A68C0018018A042E4D80020ED
:1067000030740846F8BD00004016002050C3000059
:10671000002002400548416802221143416041685F
:106720000122114341600020704700000020024018
:10673000F8B50C4C1646207C0F46012808D00120E5
:1067400020740948FFF7B0FA0025002802D006E0BF
:106750000220F8BD65613E600348FFF7A5FA257485
:10676000F8BD00004016002050C3000011484168E9
:10677000C9070BD0EFF3108172B60F4AC2600F4AFF
:10678000C26081F310884168C9070ED1416889074A
:106790000DD5EFF3108172B6094A0261094A026110
:1067A00081F310884068800701D5012070470020E0
:1067B0007047000000200240EFCDAB8905040302C2
:1067C000BFAE9D8C161514137047000010B5044918
:1067D0004A69024202D04861FFF7F6FF10BD00008F
:1067E00000040140F8B500230124A2E027469F40A1
:1067F0003A4070D04D68022D01D0122D14D1DD0821
:10680000AD002D1800952D6A5E07AC46F50E0F26DB
:10681000AE46AE406546B543AC460E697546AE40E1
:1068200065462E43009D2E624D68012D05D0022D38
:1068300003D0112D01D0122D16D185680326AC4648
:106840005D00AE46AE406546B543AC46CE68754683
:10685000AE4065462E43866046680D79BE43ED0620
:10686000ED0F9D403543456006685F000325BD4040
:10687000AE46AE430D79B446AE07B60FBE40654690
:106880002E430660C6687546AE438D68BD403543ED
:10689000C5604D68ED004BD5294D6E6B26436E6388
:1068A0009E08284DB6007519AC46AD689E07360F98
:1068B0000F27B740BD4305273F07B84201D1002746
:1068C00015E0214FB84201D1012710E01F4FB84217
:1068D00002D102270BE02BE01D4FB84201D1032764
:1068E00005E01C4FB84201D1052700E00627B7405C
:1068F0002F436546AF60184D2E684F689643FF03DF
:1069000000D516432E606E684F689643BF0300D5CE
:1069100016436E60AE684F689643FF0200D516437B
:10692000AE60EE684F689643BF0200D51643EE6036
:106930005B1C0A681546DD4000D057E7F8BD000033
:106940000010024000000140000400500008005008
:10695000000C0050001C0050000401400069084079
:1069600000D00120704742694A4042617047002AC6
:1069700001D0816170478162704700000148006862
:10698000704700000801002002480168491C0160AE
:10699000704700000801002010B508480024016875
:1069A000402211430160204600F00AF8002801D07F
:1069B000012401E000F0D0F9204610BD0020024083
:1069C00070B5054609487D210024C9000068FEF71E
:1069D0008FFB00F065FE002801D0012404E00022B6
:1069E0002946501E00F0D8F9204670BD0C01002049
:1069F00070477047F8B5394C0126A078401CA0704C
:106A00002671E08A401CE0823548008802F068FB6D
:106A1000344DE888FEF717FE3349FEF739FC334F53
:106A20003968FEF7DCFB38603148F1050068002763
:106A30000090884210DB208AFEF705FE01467F2089
:106A4000C005FEF725FC0099FEF71EFC28490860EA
:106A500028480221017001E02648077002212648DB
:106A6000FFF77CFF002809D027632048234A0168EC
:106A700023480091914212DD067011E0E888FEF78C
:106A8000E2FD1949FEF704FC216BFEF7A8FB1D4946
:106A900020638842E9DB1D491B48C860E5E70770B1
:106AA000688F401EFEF7C4FD0099FEF77BFE05D8F7
:106AB0006079002802D01648067001E0144807707B
:106AC000688FFEF7C0FD09490968FEF76BFE04D226
:106AD0006079002801D003F0ADFEF8BDC4000020AD
:106AE00064000020400D002000007A4400010020D6
:106AF000040100205B000020000400500000404022
:106B00004E0000200000F0410400FA0500ED00E016
:106B10005D000020704770B505000DD002202C46A6
:106B20002034A073284601F00DFA284600F0BEF884
:106B30000020A073607370BD012070BD7047704766
:106B400010B5044600680168C943C90708D18168C7
:106B5000C943C90704D1012141602046FFF74AFF1C
:106B600020680168C943890708D48168C943890737
:106B700004D4022141602046FFF73AFF20680168F3
:106B8000C943490708D48168C943490704D404218B
:106B90004160204600F0DEF820680168C94309071B
:106BA00008D48168C943090704D4082141602046FC
:106BB000FFF7B0FF20680168C943C90608D481689F
:106BC000C943C90604D4102141602046FFF711FFD4
:106BD00020680168C943890608D48168C9438906C9
:106BE00004D4202141602046FFF7A9FF20680168F6
:106BF000C943490608D48168C943490604D44021E1
:106C000041602046FFF79AFF10BD0000F8B5040070
:106C100005D025462035A87B002802D006E00120BB
:106C2000F8BD00206873204600F052F80220A873D7
:106C30002068C26884466368012B04D00120A16AE1
:106C4000C005814201D11E208243154861698142FD
:106C500001D0144802401448A66802401846304348
:106C6000676A266A3E433043A66A30431043012BCD
:106C700003D00122D205964203D12369E2681A4368
:106C80001043074A914205D0A2691143E2690243C9
:106C9000084610436146C8600120A8730020F8BD73
:106CA000FFFF00003F1FFFFFF8F119FF10B500685C
:106CB0000549884207D10548816B4900490881632D
:106CC0000D2000F055F810BD007C0040001002407F
:106CD00010B50068084988420CD10848816BC2048D
:106CE00011438163002201210D2000F055F80D2091
:106CF00000F048F810BD0000007C00400010024089
:106D00000068C0697047000070B502240346203354
:106D10009C730F4C2568E604354325600468E568DC
:106D2000B6123543E5600568AE6801242643AE60BF
:106D300005682E6926432E610568A96101684A61CC
:106D4000006801690422114301619C73002070BD39
:106D500000040140704700000448416B01221143C8
:106D60004163816B0204114381637047001002404C
:106D7000C106C90E01208840014908607047000023
:106D800080E100E0C106C90E012088400149086089
:106D90007047000000E100E010B501F08FFA10BD6F
:106DA00002494A6882434A60704700000070004010
:106DB000024801688215114301607047007000406D
:106DC00002494A6802434A60704700000070004070
:106DD0000548016802221143016004480169042248
:106DE0001143016130BF70470070004000ED00E0CA
:106DF0000A4B1A689208920002431A600848036915
:106E0000042213430361012906D040BF20BF20BFE5
:106E1000016991430161704730BFF9E7007000409C
:106E200000ED00E0F8B504460078544D800672D5B8
:106E3000524E0027403EB06BC00004D4B06BA90591
:106E40000843B06301274E480168C90511D40168A1
:106E5000821511430160FFF791FD009005E0FFF7F7
:106E60008DFD0099401A642837D845480068C00550
:106E7000F5D532680321090560680A400140914256
:106E800008D08103890F032904D13168890301D512
:106E90000120F8BD2A69032109040A4022D00840D4
:106EA00090421FD0207880061CD528692A69884323
:106EB0000121C9040A432A612A698A432A61286197
:106EC000C0050FD5FFF75AFD009008E0FFF756FD0B
:106ED0000099411A2B48814201D90320F8BD286945
:106EE0008005F3D561688803800F032805D13268D7
:106EF0000005824301400A43326028690322616829
:106F00001204114008432861002F04D0B16B012006
:106F100000078143B1632078C00705D0E868A16805
:106F2000800880000843E8602078800705D5E8687D
:106F30000C218843E1680843E8602078400706D5C3
:106F4000E86803218902884321690843E8602078C2
:106F5000000706D5E86803210903884361690843EF
:106F6000E8602078000606D5E86803218904884394
:106F7000A1690843E8600020F8BD0000401002400D
:106F80000070004088130000F8B50E4605007DD063
:106F900053480068C007C00FB0420AD25048016889
:106FA00049084900314301600068C007C00FB04282
:106FB00071D128784B4C800705D5E068F0218843D3
:106FC000A9680843E0602878C00752D068680228A2
:106FD00017D0032818D02168012818D08905002966
:106FE00059DAE168890889000143E160FFF7C6FCCE
:106FF00069680746022912D003291CD0012926D02E
:1070000033E021688903EAE721688901E7E7490756
:10701000E5E7FFF7B3FCC11B3348814223D8E068A2
:107020000007800F0228F4D123E0FFF7A7FCC11B63
:107030002D48814217D8E0680007800F0328F4D15B
:1070400017E0FFF79BFCC11B274881420BD8E06883
:107050000007800F0128F4D10BE0FFF78FFCC11B64
:107060002148814201D90320F8BDE0680007800F64
:10707000F3D11B480168C907C90FB1420DD9016896
:107080004908490031430160006800E003E0C0079F
:10709000C00FB04201D00120F8BD2878400706D5C6
:1070A000E068072109028843E9680843E06028781E
:1070B000000707D5E0680721C90288432969C9008C
:1070C0000843E06000F036F8E168084A0906090F55
:1070D000515CC840064908600020FFF771FCF8BD0C
:1070E0000020024000100240881300006AAA000835
:1070F0000C010020044805490068C968044A490594
:10710000490F515CC84070470C010020001002403C
:1071100083AA0008044805490068C968044A89042C
:10712000490F515CC84070470C010020001002401C
:1071300083AA000810B5184AD1680C20084004281A
:107140000BD0082810D00C2810D050680004410F34
:107150000120C003491C884010BD1068C00601D53D
:107160000E4810BD0E4810BD0E4810BD88020E4BD3
:10717000000F185C0902D368890F491CDB0301D595
:10718000084A05E01268D20601D5044A00E0044A24
:107190005043FDF7ADFF10BD0010024000093D0057
:1071A0000024F40000127A007AAA0008FEB5050057
:1071B0007ED0FE4CE7680C20E66807400120000402
:1071C00006402878C00747D0082F05D00C2F0AD1D9
:1071D00001200004864206D1206880033CD56868FF
:1071E0000028E5D038E0012069680004814203D11D
:1071F00021680143216011E0052301221B04920450
:107200009942216802D111432160F1E78143216055
:107210002168014000912068904320606868002840
:107220000DD0FFF7ABFB009005E0FFF7A7FB00993F
:10723000401A64287AD820688003F6D50CE0FFF75E
:107240009DFB009005E0FFF799FB0099401A642828
:10725000F0D820688003F6D42878800755D5092314
:10726000E868042F0DD00C2F01D1002E09D0002882
:107270003BD02168994301432160FFF77FFB06461D
:1072800027E02168490701D5002891D061681F22B5
:10729000120291432A6912021143616021689943E5
:1072A00001432160FFF746FFE16809060A0F00E08D
:1072B00079E1BF49895CC840BE4908600020FFF7FA
:1072C0007FFB002872D120E0FFF758FB801B0228CB
:1072D000B0D820684007F7D560681F2109028843AD
:1072E00029690902084360600FE0206840084000F7
:1072F0002060FFF743FB064604E0FFF73FFB801BDF
:10730000022897D820684007F7D42878C0065FD5B0
:10731000002F0CD0A869002849D02068FF21013136
:1073200008432060FFF72AFB06462DE0C0E02068F6
:10733000800502D5A8690028A7D060680721490305
:107340008843296A084360606068297F0002000A58
:10735000090608436060286A410B0120C003491CEC
:107360008840E16809060A0F9149895CC840914943
:1073700008600020FFF724FB002817D128E0FFF762
:10738000FDFA801B0228A3D820688005F7D5606825
:10739000072149038843296A084360606068297FA0
:1073A0000002000A09060843606011E0E1E021687C
:1073B000FF20013081432160FFF7E0FA064604E038
:1073C000FFF7DCFA801B022872D820688005F7D40A
:1073D0002878794E000724D568690028306910D0D4
:1073E000012108433061FFF7C9FA009005E0FFF77B
:1073F000C5FA0099401A02285AD830698007F6D594
:107400000FE0400840003061FFF7B8FA009005E057
:10741000FFF7B4FA0099401A022849D8306980076A
:10742000F6D42878400765D500200290A06BC000F4
:1074300006D4A06B012109070843A0630120029034
:107440005E480168C90511D40168821511430160C5
:10745000FFF794FA009005E0FFF790FA0099401AC0
:10746000642825D855480068C005F5D5FF20AA68CE
:107470000130824203D131690143316111E00121C0
:107480008902002A07D005231B029A4203D13269E0
:107490000A433261EFE732698243326130698843DF
:1074A0003061A86800280FD0FFF768FA009007E065
:1074B0005EE0FFF763FA0099411A4148814257D8CC
:1074C00030698005F5D50DE0FFF758FA009006E029
:1074D000FFF754FA0099411A3948814248D8306977
:1074E0008005F5D40298002804D0A06B012109077B
:1074F0008843A063686A002864D00C2F3ED0012620
:1075000036060228206805D0B0432060FFF736FA1F
:1075100005462FE0B0432060FFF730FA074604E04D
:10752000FFF72CFAC01B022822D820688001F7D46C
:10753000E96AA86AE2680843296BFD231B049A43A1
:1075400011430843E060206830432060FFF716FADB
:10755000054604E0FFF712FA401B022808D820680D
:107560008001F7D52EE0FFF709FA401B022801D968
:107570000320FEBD20688001F5D423E00128F8D067
:10758000E06801210904AA6A014091420BD10F2150
:107590008904EA6A0140914205D103218905084026
:1075A000296B88420ED00120FEBD00000010024071
:1075B0006AAA00080C010020401002400070004040
:1075C000881300000020EFE770B5040007D0002604
:1075D00025464035A662687C002802D005E00120DF
:1075E00070BD2E74204600F02FF8022068742068C9
:1075F0000168402291430160A168606822690843E4
:10760000E16811430843616901220843A1695202FC
:1076100011400843E1690843216A0843A16A08430D
:1076200021680860A0690421000C0840616A0843D1
:10763000216848602068C16992009143C161666514
:1076400001206874002070BD10B586B00446142176
:107650006846FDF7ACFD10492068884219D10F48F3
:10766000416B821411434163C16A01221143C1621B
:10767000C06A002110400590E02000900220019097
:107680000320039002910491052069460007FFF74B
:10769000A9F806B010BD0000003001400010024003
:1076A000094910B5401E884201D9012010BD074C80
:1076B00060610321081F00F001FE0020A061072087
:1076C0002061002010BD0000FFFFFF0000E000E08F
:1076D00070477047F8B502680446D069116893682E
:1076E00005072D0F5BD0DD07ED0FFF2621360E407D
:1076F0002E4367D0C60706D0CE0504D501261662F4
:10770000E26F3243E267870702220426002F06DA7F
:10771000DF0704D027683A62E76F3743E767470718
:1077200006D5DB0704D023681E62E36F1343E367CB
:10773000020709D520220A402A4305D023680822DF
:107740001A62E36F1343E367E26F002A2FD08006CB
:1077500006D5880604D5216E002901D02046884729
:10776000E06F21688968490601D4000724D52046C6
:1077700001F03AFF20688168490619D581684022E6
:1077800091438160E06E002812D020498163E06E51
:10779000FEF78EFE00280AD0E06E816B06E08506BB
:1077A00010D58D060ED5216E1CE020468847F8BD09
:1077B0002046FFF78EFFF8BD2046FFF78AFF002026
:1077C000E067F8BDC50208D55B0206D501200005BB
:1077D00010622046FFF77CFFF8BD030605D50B06B7
:1077E00003D5616E0029E0D1F8BD4006FCD54806FE
:1077F000FAD51368204640218B431360202161672E
:107800000021616600F069F9F8BD000045950008A7
:1078100010B5040003D0606F002802D007E00120FB
:1078200010BD002170200155204600F027F82420CB
:10783000606720680168490849000160204601F03E
:107840001DFF0128ECD0606A002802D0204601F01C
:107850005BFD206841680922D202914341602068A3
:1078600081682A22914381602068016801221143C6
:107870000160204601F0AEFD10BD0000F0B587B0FC
:10788000064614216846FDF792FC2C493068884270
:1078900051D12B48416B0122920311434163C16ACC
:1078A00001221143C162C06A0025104005900320E7
:1078B000400200900220032701A9A1C104200490E6
:1078C000052069460007FEF78DFF1F4C1D48A56087
:1078D000E56081C48027E560A760202025616061A4
:1078E0000002A0611848083CFEF75CFE002801D0A9
:1078F000FEF756F9F466A662144C12482146143875
:1079000020600320606010200831A1C16561A5617D
:10791000E56120462562FEF745FE002801D0FEF70E
:107920003FF9B466002201211B20A662FFF734FA5A
:107930001B20FFF727FA07B0F0BD00000038014018
:107940000010024030000240B0150020F815002061
:10795000F8B50446806F20284DD100290BD0002AAD
:1079600009D00123A0681B03984206D12069002892
:1079700003D1C80701D00120F8BD25466035287C19
:10798000012838D001202874582061650253002650
:10799000E6672220A067E06E002819D01749C1626F
:1079A000E16E17480863E16E16484863E06E1346BF
:1079B0008663676D21683A462431E06EFEF73AFE31
:1079C000002805D01020E0672E7420206067D2E7E1
:1079D0002E7420680168FF22013211430160206883
:1079E000816801221143816020688168402211432F
:1079F00081600020F8BD0220F8BD0000A1950008BC
:107A0000DF9500085995000870477047FFB5044698
:107A1000406F83B017460D4620285CD1002D0AD058
:107A2000002F08D0A168C001814207D12069002839
:107A300004D1E80702D0012007B0F0BD2046603035
:107A40000290007C012846D0029801210174002098
:107A5000E06721206067FEF791FF264640360190DF
:107A6000378277820120A1680003814202D1206918
:107A7000002802D02F46002511E000270FE0002249
:107A80008021204601F00EFF002815D1002F15D0CF
:107A90002168387888627F1C708A401E7082708AE4
:107AA000019B002806980090E9D100224021204641
:107AB00001F0F8FE002808D00320BDE728882168DF
:107AC000C005C00D8862AD1CE6E720206067029902
:107AD00000200874B0E70220AEE770470149024871
:107AE000C160FDE70400FA0500ED00E010B50524D3
:107AF0002407002204212046FEF739FF0022082136
:107B00002046FEF734FF0A2002F0CBF901220421BF
:107B10002046FEF72CFF0A2002F0C3F900220421C0
:107B20002046FEF724FF10BD10B5052424070022CF
:107B300004212046FEF71BFF012208212046FEF704
:107B400016FF0A2002F0ADF9012204212046FEF7BB
:107B50000EFF0A2002F0A5F9002204212046FEF7BC
:107B600006FF10BDF8B50024052607462546360752
:107B7000002204213046FEF7FAFE0A2002F091F9B5
:107B8000012204213046FEF7F2FE6006040E0821B1
:107B90003046FEF7E3FE002801D0641CE4B2052065
:107BA00002F07FF96D1CEDB2082DE1D3002F03D058
:107BB000FFF79CFF2046F8BDFFF7B6FFFAE770B568
:107BC000052605463607002204213046FEF7CFFE83
:107BD0000024E80901D0012200E0002208213046FB
:107BE000FEF7C5FE6806050E0A2002F05AF90122CA
:107BF00004213046FEF7BBFE0A2002F052F90022B3
:107C000004213046FEF7B3FE0A2002F04AF9641C54
:107C1000E4B2082CDDD370BD10B505242407012281
:107C200008212046FEF7A3FE012204212046FEF78C
:107C30009EFE002208212046FEF799FE0A2002F04F
:107C400030F9002204212046FEF791FE10BD10B548
:107C500005242407002204212046FEF788FE002286
:107C600008212046FEF783FE0A2002F01AF90122BD
:107C700004212046FEF77BFE012208212046FEF764
:107C800076FE0A2002F00DF910BD70B505252D070E
:107C90000024012208212846FEF769FE062002F092
:107CA00000F9012204212846FEF761FE062002F0B9
:107CB000F8F807E0641CE4B2FA2C03D9FFF7C7FF19
:107CC000012070BD08212846FEF748FE0028F1D1AA
:107CD000002204212846FEF74AFE002070BD000065
:107CE000F8B501F0A7FB01F0E1FB47480068C06967
:107CF000464E474F800700D5FE60FEF741F84549E4
:107D0000454C898F002914D044490A780121890201
:107D1000002A0AD0012A04D0022A04D0032A08D15A
:107D200003E0212801D2002200E001222046FEF7D4
:107D30001EFE0121C9023848FEF710FE384C00250E
:107D4000002824D037480560E079002803D10120BD
:107D5000E07101F0EBFD2078632806D900220821AC
:107D60002D48FEF704FE012205E0012208212A48E1
:107D7000FEF7FDFD002201210520C9030007FEF7E3
:107D8000F6FD244C4034A08C012803D01CE0E571A2
:107D90000022EBE724486946088072B68021234818
:107DA000FDF716FF002804D0022269461F48FDF7A0
:107DB000B3FF62B61EA001F057FEA58402F0D6FD07
:107DC000642002F067F8FE60608C012808D1114839
:107DD0006584058002F0CAFD642002F05BF8FE6055
:107DE000208C012806D1258402F0C0FD642002F019
:107DF00051F8FE600748124A0188914202D1C088BA
:107E0000002800D1FE60F8BD301500200400FA05FE
:107E100000ED00E0400D0020000400505B00002059
:107E2000C400002000010020AAAA0000384A00086F
:107E3000BDF8C8EBC9FDBCB6C4A3CABD0D0A00009D
:107E4000AA55000008B53721202000F06EF8032164
:107E5000212000F06AF84021222000F066F8082175
:107E6000232000F062F8AA21302000F05EF80A48D2
:107E7000008FC1B2322000F058F80221332000F008
:107E800054F85F21202000F050F8684600F006F812
:107E90000A2002F006F808BD400D002010B501468A
:107EA0000F2000F021F8002800D0012010BD10B5EF
:107EB0000446FFF7B1FE3220FFF781FEFFF7E5FE33
:107EC000E0B2FFF77CFEFFF7E0FEFFF7A5FE3320F0
:107ED000FFF775FEFFF7D9FE0020FFF743FE0446CB
:107EE000FFF7B5FE204610BD10B50C46FFF7DFFFCB
:107EF0002070012010BD70B50D460446FFF78CFEC2
:107F00003220FFF75CFEFFF7C0FEE0B2FFF757FE3E
:107F1000FFF7BBFE2846FFF752FEFFF7B6FEFFF75E
:107F200096FE0A2001F0BDFF70BD10B5FFF7E3FF1C
:107F3000012010BD10B50248FEF702FE10BD000082
:107F4000A8140020FEB50446002572B60068394A20
:107F5000831804D13849CD68032189040D40816814
:107F60000191C168009141698669002B08D13248AE
:107F70004038836AC7043B438362836ABB4383629E
:107F80000846304348D02B482368C34205D12A48CD
:107F9000C368032292049343C360002917D020686A
:107FA000026901231A43026120684161FEF7E6FC81
:107FB0000746FEF7E3FC2168C01B0968090703D4E4
:107FC0007D21C9008842F4D9216808204860002E2C
:107FD00017D0206801690122114301612068866180
:107FE000FEF7CCFC7D270646FF00FEF7C7FC2168A4
:107FF000801B0968C90601D4B842F6D9216810204F
:1080000048600C482168C14206D10B48C168032270
:10801000920491432943C1602068016949084900DD
:10802000016121680198886021680098C86062B683
:10803000FEBD00000084FFBF401002401CB50021BF
:1080400016480091144A01910260C1631205426012
:10805000816007228263012202610246C1602032F0
:108060001170FF235170C233436281621173016347
:108070008161042241634261C161FEF77FF80848D3
:1080800000908013019069460448FEF727F800210C
:108090000248FDF7CDFF1CBD002401404C14002018
:1080A0000200000408B50848016B01221143016376
:1080B000006B01211040009000220A20FEF76CFEA8
:1080C0000A20FEF75FFE08BD00100240F0B587B041
:1080D00014216846FDF76BF84C48C26A04210A4334
:1080E000C262C26A0A400592C16A80273943C162EE
:1080F000C16A39400591C16A01252943C162C16A3B
:1081000029400591C16A02263143C162C06A2A46EC
:108110003040059005201C210007FEF728FC0122B5
:108120003B493C48FEF723FC00223B493948FEF717
:108130001EFC91210520002209020007FEF717FC12
:1081400036480190002405206946009502940007F6
:10815000FEF748FB03200190052069460096029433
:108160000007FEF73FFB0C20009011200190032038
:1081700003900520029469460007FEF733FB1020A8
:108180000090052069460396019502940007FEF7CA
:1081900029FB1120019002946946009503941D4823
:1081A000FEF720FB1E48019069460096029519488B
:1081B000FEF718FB1B480090029469460195039452
:1081C0001448FEF70FFBE8026A4651C2694611489F
:1081D000FEF708FB912000020090052002946946FA
:1081E000019503940007FEF7FDFA694609480097D8
:1081F00002950194FEF7F6FA002201210520FEF710
:10820000CBFD0520FEF7BEFD07B0F0BD001002401B
:1082100001060000000400500830000000001110AA
:10822000000021100836000010B50F4C0D482060EA
:10823000FF20053060600020A060E0602061606188
:10824000E0610121206249026062A161A062072011
:10825000E0622046FFF7B8F9206801684022114328
:10826000016010BD00300140D814002000B585B079
:1082700014216846FCF79BFF0E480D490160E1217F
:108280004902416000218160C160016181610C226D
:10829000C1614261016230214162012109038163B0
:1082A0004900C163FFF7B4FA01F03AFB05B000BD25
:1082B0000038014030150020704700008307FF227E
:1082C000DB0E9A408907090E994000280BDA000757
:1082D000000F0838830808489B001818C3699343A7
:1082E0000B43C3617047830804489B001B18186840
:1082F000904308431860704700ED00E000E400E0A0
:10830000BFF34F8F04490348C860BFF34F8F00BFCE
:10831000FDE700000400FA0500ED00E0F0B58DB0C7
:108320000A2002F09BF87D20C00002F0B1F8F84C62
:108330000025A570E07B0C2801D30B20E0730122FF
:10834000052051020007FEF712FB0026F148E670F7
:10835000F14D00782871F149A0790978400008436F
:10836000617D89000843E871E06AE870401CE062C2
:1083700060792946A8744200B4310846A138FCF758
:10838000FDFE06206872E648E14A0078A872207F68
:10839000287328461338917F0175D17F4175607924
:1083A000002240002946153002F042F96079002190
:1083B0004000153002F04EF9022002F09FF8EE71F5
:1083C0006674E672012060732673D648FEF798FC47
:1083D00060840546E6706079FDF750F9D24AD34BC8
:1083E000FDF746F801F0F2FC012300229B07FCF7A1
:1083F0008DFFFDF789F90006C00C401980B20121FC
:10840000C903A084884201D3401AA084C848A0634D
:108410002079401C2071C348FEF772FC2084BE48BE
:10842000C44E4E300690A9E1BE48FEF769FC208498
:10843000C14F25460AE0BB48FEF762FC80B22884A3
:10844000A98C884202D38919884206D300210F20C3
:1084500001F084FF38422863EDD0286B411C20D006
:1084600040047DD58122D20100210F2002F0B5F811
:108470007D20C00002F00CF8002001F0BEFF0021BA
:10848000102001F06BFF4106A348490E0022503036
:10849000A96401F099FFA0485030417A0729C2D160
:1084A00001E0FFF72DFF07460222A449401DFCF71B
:1084B00089FE0028B7D102F01EF96965286502F02F
:1084C00007F9E965A865E8786946401CE8709248B4
:1084D0004D3002790A70407948700888E98B8842EB
:1084E0007ED106989649008A08808B4888494C308E
:1084F000808A48838B48FEF703FC2884688B914967
:10850000FF30C33080B2688388420DD94942401899
:1085100068838B488B4A01880B32491C89B20180E1
:10852000914201D3002101800698794A8189918680
:10853000C089D0866A6BAA63FB7C1A07120F032AD4
:1085400000D0EA741A0900232A752B710127704B99
:10855000EF7219875887002A14D00222774900E069
:10856000FFE06D485530FCF72DFE00280AD16A491E
:108570006F74CF71A86C64311638C2B2AA74724895
:10858000FCF7FCFD01202873634961480422513146
:108590004430FCF7F3FD6048EB6D1630AA6D02F035
:1085A0007FF867487D210088C90007464843698BEA
:1085B0004018E863079065483021007828740090DF
:1085C000634800884843FDF73EF8019038460A2189
:1085D0004843FDF738F80199FCF75AFE7F2100E087
:1085E0002FE0C905FCF7FBFDFDF756F881B25748AF
:1085F00001800098401E814201D101202873EF8440
:108600001620285EFDF726F805910490288CFDF7CA
:1086100035F8504A504BFCF72BFF0746039107985B
:10862000FDF718F83A46039BFCF714FF059B049AE4
:10863000FCF76CFEFDF744F82864A88B00F050FDB1
:108640009CE0FDF785FB07463F4803210C38C155E8
:1086500006992F488A898286C989C1863A4AB80014
:108660009C3A696B11502C49EB6D40181A30AA6D79
:1086700002F016F868797F1C87427FD101F08CFDEB
:10868000FF22A16D5204E06D0023891858410006B5
:108690000D0A054368084000010E0002616620666D
:1086A0001D48636D0A30226D01F0FAFF1A48636EAF
:1086B0001230226E01F0F4FF1749082048726079E9
:1086C000002280001C3001F0B3FF6079002180009F
:1086D0001C3001F0BFFF284601F0B9FE012001F077
:1086E0000DFF607202211D48FEF738F9002806D000
:1086F00000210A480170607A002802D046E001217A
:10870000F7E700210F2001F029FE0006F9D53DE032
:1087100048000020C4000020B4110020FC0000200C
:10872000D4000020A8140020B81E85EB51B8CE3F1D
:10873000A0860100983A000000D02724E400002021
:10874000F8000020E703000034130020DA000020C6
:10875000DE000020F853E3A59B843E400004005057
:108760000CE03A4600210F2001F037FF6879E978E4
:10877000401C814202D0002001F03FFE218CA08CE1
:10878000814200D250E680198142FBD801F004FDFD
:10879000664A00210F2001F020FF0021E173637978
:1087A0000846049320E0624D2A5C002A1AD0E67B3A
:1087B0008D00761CE6735E4EAC46303E72515C4DC9
:1087C0004600C03D4F00AE5B1835EE5386001835AD
:1087D000574FAE596546603F7E51491C544D521E5D
:1087E000C9B22A54401CC0B29842DCD3E0780328B6
:1087F00001D2E07BE0734F490022C87B8873401EA2
:1088000032E000212CE04A4C8B00603C1E19B4463B
:10881000E5587668B54221DD0695454D4C00A83DEA
:108820002D5B9700AE46424D303DED590595404DCC
:10883000603DEE50483D66190B9675883C4EA83E4B
:108840003553344678341F197D68E5506346069DDC
:108850005D600B9E75467580059D7D60491CC9B2A3
:108860008142D0DB521CD2B28242CADB304860382F
:1088700002683048816B32398A421BDA2C49303920
:108880000968002916D0C179491CCAB2C271032AED
:1088900005D9274AA83A1288C283022202700179B8
:1088A000032901D901210170214C00210278C03C2B
:1088B000049B09E00021C171F1E74D00655B002DCB
:1088C00000D10222491CC9B29942F6D30270184B5A
:1088D0000021194A903B8C00491CC9B21A510C293D
:1088E000F9D3407C002806D011490C310B78487828
:1088F0008A78022B0ED00D4A002180320F2001F021
:108900006CFE01210520002249020007FEF72FF826
:108910000DB0F0BD094BC91C1818FCF72FFC02F074
:1089200025F8642001F0B6FABBE5000000D027244A
:108930002813002048000020FFFF0100400D002008
:1089400070470000F0B58DB0B54801900020C043DD
:108950000A9000260A2001F081FD7D20C00001F070
:1089600097FD0020AF4C0546A070AF4FAF480B906D
:10897000AE480022C23885730146142001F058FE2B
:108980000021142001F066FE022001F0B7FD002155
:108990000F2001F0E3FC38422063F8D0206B411C2B
:1089A00018D040047ED58122D20100210F2001F091
:1089B00014FE0021102001F0D1FC41069B48490E15
:1089C0000022801C01F000FD9848801C417A022999
:1089D00002D005E1FFF794FC944802229449C01D9F
:1089E000FCF7F0FB0028F4D101F085FE61652065FD
:1089F00001F06EFEE165A065002E23D10B988D4934
:108A0000008A088089488749801E808A4883012619
:108A10008948FEF775F92084608B8849FF30C330A0
:108A200080B2608388420DD94942401881496083F1
:108A30000888824A401C80B20B320880904201D3E1
:108A4000002008800B9968468A890280C989418084
:108A500076490422C91C0846A238FCF78FFBFF2286
:108A6000A16D5204E06D0023891858410006090ADF
:108A700001430846029101F0EAFC029948084000CF
:108A8000010E0002616620666848636D9638226DAB
:108A900001F006FE6548E36D9238A26D01F000FE1C
:108AA000624800E09EE08E38636E226E01F0F8FDB1
:108AB0005E490022A0393C2001F0BAFD00213C2093
:108AC00001F0C8FD012001F019FD6072A0780121BC
:108AD000401CA0700520C9030007FDF74DF955485B
:108AE0007D220088D200014602905043628B0A39F1
:108AF0008018E0630C90524800782074049008B20B
:108B00002085002803DA7D21C900401820854D48C2
:108B1000302100884843FCF796FD05902820205E10
:108B2000FCF786FD0599FCF7B3FB7F21C905FCF72F
:108B300056FBFCF7B1FD424980B208800499491EFA
:108B4000884201D1012020730298E0841620205E23
:108B5000FCF780FD05910690208CFCF78FFD3A4ACA
:108B60003A4BFCF785FC079104900C98FCF772FDDA
:108B7000079B049AFCF76EFC059B069AFCF7C6FB64
:108B8000FCF79EFD2064A08B00F0AAFA00990198E2
:108B900081420DDA00290BD024490422C91C0AA8FD
:108BA000FCF7ECFA022020700520A07200980190DA
:108BB000607A002805D100210F2001F0CFFB0006CC
:108BC000F9D5802200210F2001F007FD00206D1C47
:108BD000EDB26070032D00D2CAE6002E08D01AE074
:108BE0000120F4E71A4A00210F2001F0F6FCF7E714
:108BF000A08B1849401E0004000CA08302D00A88F4
:108C0000904201D90888A0831349A08B0988401E8F
:108C10004843124908800A98E0830DB0F0BD000077
:108C20003F420F004800002000D0272402120020FD
:108C3000E4000020F8000020A8140020E703000052
:108C4000DA000020DE000020F853E3A59B843E40BC
:108C500000902724D0000020CE000020CC0000206F
:108C6000F8B532493048086001F020FE4120304C10
:108C7000C0006080E088002801D16420E080208F5F
:108C80000A2801D902202087E08E3C2801D93C2007
:108C9000E086284980B20870274DE08F6871A08F68
:108CA000A871A07AE870A68805212E626981E788FC
:108CB0003846FCF71DFAA88101463046FCF718FA41
:108CC0008800081886B27D20C0002E817043FCF712
:108CD000D5FC1A4A1A4BFCF733FCFCF715FDE8816A
:108CE0007D206E823946C000FCF702FA28820146D8
:108CF000C820FCF7FDF968830120E882FDF740F801
:108D0000A882EA890F491048FDF7FEFF0FA0296AE3
:108D100000F0AAFEE18811A000F0A6FE218914A0AF
:108D200000F0A2FEF8BD00005999000844000020A0
:108D3000400D002000000020C4000020F853E3A5EF
:108D40009B843E40FF7F0000A8140020B1EAC7A921
:108D500049443A202564202E0D0A0000CDA8D1B642
:108D6000BCE4B8F43A202564206D732E0D0A00008F
:108D7000B5A5B4CECDA8D1B6BBF9D5BECAFDC1BF8D
:108D80003A202564B8F62E0D0A000000F0B5904D8B
:108D900085B0012028808F4FC8208F4C3880207AE2
:108DA000401C2072C00706D0A08B411EA183022860
:108DB00001D2C820A083A08B00F092F90A2001F014
:108DC0004DFB7D20C00001F063FB02218348FDF7CD
:108DD000C5FD002838D00020814980000978824EE6
:108DE000490008437F4909780843B0721020707227
:108DF0007E48C1887D20C000FCF77AF970737C48FA
:108E00007A490078B07330460B308A780270C9789E
:108E10004170411C75482030027ECA70407E087146
:108E200072482230027E4A71407E887100220C39DD
:108E3000152001F0FDFB0021152001F00BFC0220A4
:108E400001F05CFB6B4E03E00120C5E7FEF748FF35
:108E500000210F2001F082FA30422063F6D0206B0F
:108E6000411C7DD040047CD58122D20100210F20FD
:108E700001F0B3FB0021102001F070FA41065A48BE
:108E8000490E00225030A16401F09EFA564E503631
:108E9000707A112865D102225749701DFCF792F9AA
:108EA00000285ED1F01E027969460A704079487048
:108EB000B17A2980C820FCF71BF93880307BA08369
:108EC0004E4DB01E008A28804349301F808A488357
:108ED0004B48FDF715FF80B220840390608B494911
:108EE000FF30C33080B2608388420CD949424018B9
:108EF000608328884349401C80B20B312880884217
:108F000001D3002028802D887D20C000618B68431C
:108F10004018E06302903C48067828460A3800B2C0
:108F200026742085002803DA7D21C9004018208599
:108F3000388830214843FCF786FB07462820205E0E
:108F4000FCF776FB3946FCF7A3F97F21C905FCF74E
:108F500046F9FCF7A1FB2C4980B20880761E01E09F
:108F600034E031E0B04201D101202073E5841620C5
:108F7000205EFCF76FFB074601910398FCF77EFB30
:108F8000224A234BFCF774FA05460E460298FCF77A
:108F900061FB2A463346FCF75DFA3A46019BFCF733
:108FA000B5F9FCF78DFB206468460088E0830E4825
:108FB0000D495030807C6071420063310846513069
:108FC000FCF7DCF80320207005B0F0BDFFF798F93E
:108FD000D4000020DE0000204800002000040050E3
:108FE000C9000020CA000020B4110020400D00205C
:108FF0000000002000D02724E4000020F80000201A
:10900000A8140020E7030000DA000020F853E3A5CD
:109010009B843E4070B586B014216846FCF7C7F8C3
:1090200001250F4EED03002229463046FDF79FFC37
:109030000120002401900294694600950394304673
:10904000FDF7D0FB0320019002946946009503943C
:109050003046FDF7C7FB022000F01CFF06B070BDD4
:109060000004005070470000F8B5044600206A462E
:109070001080194D55222A70AA226A700322AA7004
:10908000661DEE702A716971144A49008918AC7125
:109090002246E81DFCF772F8002007E029186A460E
:1090A0008978128889186A461180401CB042F5DB25
:1090B000611DA81CFCF7BEFC014668460180291909
:1090C0000078C87168464078087221460931024824
:1090D00000F0A2FAF8BD0000E8130020400D0020C7
:1090E00010B51A4CE08A228A6178904201D3801A26
:1090F000E08280B2628B034653435B1823831328BC
:1091000002D1424350182083208B302148436421F0
:10911000643048430E49E0620968401AA062FCF7D7
:1091200099FA0C4A0C4BFCF70BFAFCF7C9FA0B49FD
:109130006062884202DD4A4280186062002801DADB
:109140004018606206490968486110BDC4000020EB
:1091500088000020F853E3A59B843E40FF7F000079
:10916000A8140020034A1168382389B299430143A7
:10917000116070470030014010B5FDF705FC10BDCF
:1091800010B59AB034216846FCF711F814210DA8E7
:10919000FCF70DF81C2112A8FCF709F81B48016820
:1091A0000324E402A143C21489180160FDF700FE04
:1091B00017480169A143016106200090FF2001309A
:1091C0000290012003901020049002200990400496
:1091D0000B90000100240C900A946846FDF7E6FF0E
:1091E0000F200D9003200E900F94109401211194E4
:1091F0000DA8FDF7C9FE812012900320800418906D
:10920000149412A8FDF70EFE1AB010BD00700040B5
:109210004010024010480168821511430160C16886
:109220000E4A1140C16001680D4A11400160816819
:10923000490849008160016801229204914301605C
:10924000C168FD2212049143C160002101610649F9
:109250000448886070470000001002400C40FF88FE
:10926000F6FFF6FE0050000800ED00E070B501F0DA
:1092700089F8234C234DE06402E001F083F8E064B8
:10928000A842FAD1207801260525F6032D070028EB
:1092900006D001280CD0022817D003282CD129E0B1
:1092A000012231462846FDF762FBFFF76FFD06E01D
:1092B000012231462846FDF75AFBFFF743FB002207
:1092C00031462846FDF753FB16E0A07A0122401EE6
:1092D000A07231462846FDF74AFBFCF76DFD0022DF
:1092E00031462846FDF743FBA07A002804D101202F
:1092F000207001E0FFF712F800F036FF70BD0000AB
:10930000480000203001CADE10B5818CC90707D0A3
:1093100001684A6801235B049A43836A1A434A60DE
:10932000818C890707D501684A6801231B049A4389
:10933000C36A1A434A60818C490707D501684A68A5
:1093400001239B049A43036B1A434A60818C0907EB
:1093500007D501684A680123DB039A43436B1A432C
:109360004A60818CC90607D50268916801231B03F6
:109370009943836B19439160818C890607D50168F5
:109380008A6801235B039A43C36B1A438A60818C0A
:10939000490612D503685A6801210905046C8A43FD
:1093A00022435A60026C8A4207D102685168032343
:1093B0005B059943436C19435160818C090607D5BD
:1093C00001684A680123DB04806C9A4302434A60C7
:1093D00010BD0000F8B500260446C667FDF7CEFABA
:1093E000054620680068124F000709D501212B4669
:1093F000002249052046009700F054FA00280DD1BC
:109400002068006840070BD501212B460022890502
:109410002046009700F046FA002801D00320F8BD4E
:1094200020206067A067603426740020F8BD00002B
:10943000FFFFFF01F8B5184CC826E078002829D1B5
:109440006079002826D101206071144D686B0027D7
:1094500000281ED0686BC821081A15E01048E16882
:10946000405C616988470F480A21008848430E49DB
:109470000880E068401CE060E068C82800DBE76026
:10948000696BC820401A761EE168814201D0002E27
:10949000E4DC6771F8BD00003000002000000240ED
:1094A000780C0020D4000020E000002070B5224C91
:1094B000E07800283FD1207900283CD1012020719C
:1094C0001E4EF16900250906002933DA215662573C
:1094D00091420AD1F06940062CD5A079002829D004
:1094E000A5712089401C208124E0A179002903D1A5
:1094F000A0710A2000F0D5FC00202056CC21484362
:109500000F494218206912181279B262401C0022D9
:109510002061A256CC235A43895881420ADC256136
:109520002078401C207020780E2800D12570A0786B
:10953000401CA070257170BD300000200038014033
:109540005001002010B5806A0022014640314A8354
:109550004A82FEF7BEF810BD70B5846A606FA56FD1
:109560002168896800260906002906DA212804D125
:1095700052200653204600F047F8206880684006D5
:1095800006D5222D04D15A200653204600F02CF88F
:10959000E06F10210843E0672046FEF79AF870BD9F
:1095A00010B501460968806A0968890614D400224A
:1095B0005A210A5201680A68FF2301339A430A605C
:1095C00001688A68520852008A6001688A684023EC
:1095D0009A438A6020218167FEF716FA10BD10B504
:1095E000806AFEF712FA10BD01680A68FF23213372
:1095F0009A430A6001688A68520852008A602021F2
:10960000816700210166704701680A68C0239A4398
:109610000A6020214167704770B5164CE278002A35
:109620000CD12279002A09D10122E2700025C82933
:1096300003DC0222A256002A01DCE57070BD012382
:10964000E356CC2253430C4AD1500123E356CC2697
:1096500073439B180A460146181DFBF78FFD60787F
:10966000401C607060780E2800D16570A078401EA4
:10967000A070E2E73000002050010020F8B5044659
:109680002669A268E76932436669102000253E43D7
:109690002368324378491E68784F3E4016431E6067
:1096A00023685A6803263603B243E66832435A6099
:1096B0002368A2698B4201D0266A32439E680B2739
:1096C0003F02BE4316439E606D4E23686D4AB3420F
:1096D0000CD1D2689207920F06D0012A38D0022A04
:1096E00034D0032A20D11EE001201DE0664EB34293
:1096F0000AD1D2680C26324026D0042A28D0082A63
:1097000024D00C2A10D10EE08B420DD1D668032252
:109710009202164018D001229202B61A18D0B61A38
:1097200014D0964200D10820564A0126403A574F9D
:10973000F6038B4236D100280CD002280DD0042825
:1097400012D008281FD11CE00020EDE70220EBE733
:109750000420E9E7FDF7CEFC08E01068C00601D55B
:10976000384605E04A4803E0FDF7E4FC002873D0E2
:10977000626851005118814205D81103814202D319
:1097800003E03046F4E7012566E0010E06025008CA
:10979000002330185941FBF7C1FC03210902411A8B
:1097A0003C4A55E0E169B14232D1030000F083F94F
:1097B00009070A0D06250606062B0600E3E7FDF756
:1097C00099FC1CE0FDF7A6FC19E010686168C00672
:1097D00002D54808304A01E0304A48088018FBF7B3
:1097E00087FC80B201462E4A10399142CBD8511CD9
:1097F00001400007400F08432CE0FDF79BFC616827
:1098000040004A08EAE76168012248081204E5E7D7
:10981000030000F050F909070A0D06260606062C7B
:109820000600B0E7FDF766FC1DE0FDF773FC1AE0EB
:1098300010686168C00602D54808C01902E01448E3
:109840004A081018FBF754FC80B20146144A10393C
:10985000914298D82168C86000202066606628463A
:10986000F8BDFDF767FC61684A088018EAE761689F
:1098700048088019E6E7000000480040F369FFEF60
:1098800000380140401002400044004000093D0003
:109890000024F400FFFC0F0000127A000048E801E9
:1098A000EFFF0000FFB581B017460E4604460A9D43
:1098B00009E0681C07D0FDF761F80499401AA84236
:1098C0000CD8002D0AD02068C1693046884318D0D2
:1098D0000020B842EDD0002005B0F0BD206801683E
:1098E000FF22A13291430160206881684908490044
:1098F000816020206067A06700206034207403200E
:10990000EAE70120E5E7000010B5044910200968E6
:1099100008620248FDF7DEFE10BD00003015002091
:1099200001490D20887070473000002010B50748AD
:109930000A22018A51438183FEF7B4FBFEF796FCAD
:10994000C82203490348FEF703F810BDC4000020F5
:10995000780C002030150020F8B53E4C002321780B
:109960003D4A1D46082910D0072947D0062950D066
:10997000052952D0042953D0032954D0002956D0A8
:10998000012958D002295AD05BE0A17800264A1F4D
:1099900004E0314FBF5DFB189BB2761C9642F8DBAA
:1099A000667927799A195118E3786278C918891865
:1099B000C9194018C0430006000E1AD1012E14D058
:1099C000022E16D125482449C018FBF7D7FB00F01A
:1099D000CDFF642000F05EFABFF34F8F214920488D
:1099E000C860BFF34F8F00BFFDE759081046FFF76F
:1099F0003BFB2570E570A570A571F8BDA1795054A9
:109A0000491CC8B2A071A178491F8842F5D108202D
:109A100001E0607007202070F8BDE0700620FAE7D2
:109A200060710520F7E7A070E5700420F3E7552882
:109A300007D10120EFE7AA2803D10220EBE7032892
:109A400003D02570E570A570F8BD0320207020714B
:109A5000F8BD0000BB00002084130020400D002052
:109A60000400FA0500ED00E00FB410B503A9044BA3
:109A7000044A029800F002F910BC08BC04B0184770
:109A8000B9A60008100100202021020C01D01021ED
:109A90001046020A01D010460839020901D01046CA
:109AA000091F820801D01046891E420801D0881E75
:109AB0007047081A704730B47446641E2578641CD9
:109AC000AB4200D21D46635D5B00E31830BC184713
:109AD00002E008C8121F08C1002AFAD17047704777
:109AE000002001E001C1121F002AFBD1704708B518
:109AF0000021684601706B46012202212C2000F0F3
:109B00007BFD0221684601706B4601222C2000F08B
:109B100073FD08BD38B504466D20694608706B4674
:109B2000012207492E2000F067FD0649002C01D0D4
:109B3000054A00E0054A2E2000F044FD38BD000033
:109B400006080000061800000706000007160000BF
:109B500038B504466B4602220021362000F018FC7E
:109B6000B3212300FFF7A7FF0E0F08153A3A3A3A40
:109B70001C273A3A2F34483A002168460170407851
:109B80004108490014E06946087880088000401CBC
:109B900004E06946087880088000801C08701DE099
:109BA000684602780A4048320270417880200143BA
:109BB0006846417012E0684602780A4002704078B8
:109BC0004106490EF4E7694648780221084303E05C
:109BD00069464878FD210840694648706B46012275
:109BE0000021362000F008FD012200AB114636208E
:109BF000013300F001FD38BD69460878CF210840E7
:109C000069462030CAE708B5032168464170012142
:109C100001706B4602220021362000F0EDFC01228B
:109C2000D20306212D2000F0CDFC012000F032F9F6
:109C30000120FFF78DFF08BD08B5020A69464A708A
:109C400008706B46022204212D2000F0D5FC032071
:109C5000694608706B46012206212D2000F0CCFCDD
:109C60000020694608706B46012206212D2000F075
:109C7000C3FC0A212D2000F071FB08BDFFB58DB09B
:109C80000446002506E025280AD0109A0F9990472F
:109C9000641C6D1C20780028F5D1284611B0F0BD59
:109CA00000270121484A009700E00743641C2378FD
:109CB0000846203B98401042F7D120782E2817D133
:109CC000042007436078641C2A280CD10E98641C79
:109CD00002C800910E900BE000990A2251433039DE
:109CE0004018641C00902078014630390929F3D9C6
:109CF00020780028D1D0642808D0692806D075289B
:109D00001ED0109A0F9990476D1C5BE00A200E99A7
:109D1000019001C90E91002802DA40422D2102E093
:109D2000390504D52B216A461172012103E0F90798
:109D300004D02021F7E70BAE0B910DE00021FAE7EC
:109D40000A200E99019001C90E91F7E70199FBF7DE
:109D5000CFF93031761E31700028F7D103A8801B6F
:109D600020300190780701D5009801E00120009093
:109D70000199884201DD401A00E000200027009090
:109D800006E002A8109AC05D0F9990476D1C7F1CD9
:109D90000B988742F5DB04E0109A30200F9990472A
:109DA0006D1C0099481E00900029F5DC05E0307814
:109DB000109A761C0F9990476D1C0199481E0190CE
:109DC0000029F4DC641C65E709280100F8B54A00A5
:109DD0002B4B520DD6182B4A0C460546142E2BDA67
:109DE000002E12DA284BFBF791FA00221346FBF7FC
:109DF000B7FD40D2002C03DA0124E40700253AE045
:109E00002046284337D0214C14E0214F0B46F74021
:109E10003B402B4331D01C4BFBF778FA0022134612
:109E2000FBF79EFD27D2002C03DD01200005F0404A
:109E30000419BC4300251EE0332E1EDC33460027E8
:109E4000143BFF43DF40384217D00F4BFBF708FBB2
:109E500000221346FBF784FD0DD2002C0ADD142EE0
:109E60000CD03420811B012088404019A84200D228
:109E7000641C0546BD4321462846F8BD641CF9E72D
:109E800001FCFFFF9C7500883CE4377E0000F03F3A
:109E9000FFFF0F007D2110B5C900484300F001F815
:109EA00010BD002140E000BF00BF00BF00BF00BFE9
:109EB00000BF00BF00BF00BF00BF00BF00BF00BFAA
:109EC00000BF00BF00BF00BF00BF00BF00BF00BF9A
:109ED00000BF00BF00BF00BF00BF00BF00BF00BF8A
:109EE00000BF00BF00BF00BF00BF00BF00BF00BF7A
:109EF00000BF00BF00BF00BF00BF00BF00BF00BF6A
:109F000000BF00BF00BF00BF00BF00BF00BF00BF59
:109F100000BF00BF00BF00BF00BF00BF00BF00BF49
:109F200000BF00BF00BF491C8142BCD37047000086
:109F3000FEB504460020019000906079734940000E
:109F40000E5A61782578491E7148CFB20163042DFD
:109F500077D0072D75D000210291217801736C49CB
:109F6000E379012292058969002B6CD091438161CC
:109F70006748217A4173217A82698907890B0A43EC
:109F800082610021042000F028FB324661492E2026
:109F900000F018FB3846FFF7BDFD5F4E0522705DEF
:109FA000810040185D49431807212B2000F024FB55
:109FB0005B49029801220B180B21282000F01CFBA2
:109FC000705D584980000A580C21282000F005FBDC
:109FD000E079554980004018A1794900425A022190
:109FE000272000F0EFFA51487E00825B04212720F1
:109FF00000F0E8FAE079002829D0A07804282CD0D5
:10A0000028206946087220220621272000F0DAFA6B
:10A0100002AB01222621272000F0EEFA4449380144
:10A020004018E178890042580821272000F0D5FA2D
:10A03000A17A601C627A0902114313D016E000E095
:10A0400001E0012188E71143F608816190E764226D
:10A050000621272000F0B6FAE0E7102069460872D2
:10A060000246D1E733490172090A4172417A007A06
:10A070000A0202432021272000F0A4FA2E4F0C21CF
:10A0800023203A6800F0A9FAF019828804212320DD
:10A0900000F098FAA07900280BD0E0792749012236
:10A0A00043180021212000F0A7FA0320019001208D
:10A0B00000902A07120F10010243607800218007E8
:10A0C000000B02430198000502430098400402433C
:10A0D0002079C006400902436079C00602431F2070
:10A0E00000F07BFAA0786178012308430204084855
:10A0F000DB030261E179490319430A43026100214C
:10A10000082000F06AFA0020FEBD000038AA00080E
:10A110001401002004280000E0A90008010000202C
:10A120001F000020E8A9000808AA000814AA0008D7
:10A1300018AA00084110000000AA00082100002011
:10A1400038B50C4607498A8B002102432C2000F0C9
:10A1500039FA684604706B46012206212C2000F073
:10A160004BFA38BD1401002010B5FFF7C0FC10BD3C
:10A1700010B504460421362000F0F0F80121C90290
:10A18000002C01D0084300E0884302460421362019
:10A1900000F023FA10BD000038B540206946087071
:10A1A00000210E2000F0DAF80446002211460E20AD
:10A1B00000F013FA6B46012200210D2000F01CFA7A
:10A1C000074A00210F2000F008FA00F0E1F92246CA
:10A1D00000210E2000F001FA02480021017338BD71
:10A1E000F8FF2724340100207CB505460420694689
:10A1F00008704B4C00206075214620312063487167
:10A200000873A0836063A06300F0BCF8454E206033
:10A2100002E000F0B7F82060B042FAD10020FFF76A
:10A2200097FC41480078242801D9243806E006210B
:10A23000FAF75EFF0622101A4001084302060104E5
:10A240000A4301020A43024300211E2000F0C5F91F
:10A250006B4601220021242000F0CEF91E20FFF7DA
:10A26000EBFC86B2300AA0730420FFF7E5FC000681
:10A27000000E0DD002206946087101AB01221221A7
:10A280002D2000F0B9F9A08B012109030843A08318
:10A2900000F078F820600620FFF7CEFC6060072011
:10A2A000FFF7CAFCA060F006C00E207501D1102097
:10A2B0002075C0B200F0DCF9E80707D0FFF7A3FC77
:10A2C000A08B0121C9020843A0830AE005213620A2
:10A2D00000F02EF81549084002460521362000F00E
:10A2E00071F90120FFF734FC0021042000F036F85A
:10A2F000A0610021262000F031F8152189030843D0
:10A3000002460021262000F068F90022262136208E
:10A3100000F058F900F036F8206000207CBD000005
:10A32000140100203001CADE00000020FFFD000003
:10A3300038B5094C89B280B26B46022200F028F889
:10A34000002806D16846407801026846007808185F
:10A3500084B2204638BD0000FFFF000038B500245D
:10A36000E44389B280B26B46042200F011F8002861
:10A3700006D103216846435C2202D418491EFAD54F
:10A38000204638BD10B500210846FFF7E7FF10BD95
:10A3900038B5002909D0402420436C462070C8B24B
:10A3A0007F2906D8607002200AE069460870012003
:10A3B00006E0802420436C466070C809A07003202A
:10A3C000694600F0ADFA38BD10B5144603460A469A
:10A3D00021461120FFF7DCFF10BD10B50346052212
:10A3E00000211520FFF7D4FF10BD10B5034605224C
:10A3F00000211720FFF7CCFF10BD38B5054600201F
:10A400006946087000F0C4F8FF2401342246002D8C
:10A4100001D00322120200210D2000F0D3F8002DFC
:10A4200013D06B46012203210F20FFF7B1FF6846CE
:10A430000078000709D5FFF7AFFE224600210D2066
:10A4400000F0C0F80020C04338BD002038BD10B572
:10A45000024601210A2000F0C0F810BD10B50446E4
:10A4600000211A20FFF77AFF000D22030005120BCE
:10A47000024300211A2000F0B0F810BD10B50246CA
:10A4800002492E2000F09EF810BD000004180000C4
:10A49000F8B505466B46012203210420FFF778FF3B
:10A4A0000126114C3607002D0DD02A4600210C2024
:10A4B00000F088F86946087810210843694608705A
:10A4C000A069304307E069460878EF2108406946F3
:10A4D0000870A069B0430B46A0610122032104204B
:10A4E00000F08AF8F8BD00001401002010B5024603
:10A4F0000021182000F066F810BD0000F8B50746EE
:10A50000002568460570B807204C2E4600280ADA58
:10A510008020694608706B46012200210D2000F062
:10A520006BF801202073F8076946087821D00621CE
:10A530000843694608706B46012200210D2000F097
:10A540005BF803210F20FFF7F3FE8121C9000842C9
:10A5500019D04020694608706B46012200210D2069
:10A5600000F04AF80020FFF703FE00252673ED43B4
:10A5700009E002210843694608706B460122002168
:10A580000D2000F039F82846F8BD00003401002005
:10A590001CB56B46012203210F20FFF7F9FE684628
:10A5A00000784022C1091040C9014000814208D012
:10A5B000012069460871024601AB03210D2000F01D
:10A5C0001BF81CBD08B56B461A70120A5A7089B286
:10A5D00080B2022200F010F808BD38B500236C46A6
:10A5E000E254120A5B1C042BFADB89B280B22346C8
:10A5F000042200F001F838BD38B58024002909D0C4
:10A60000C02528436D462870C8B27F2907D86870D6
:10A61000022009E0204369460870012004E020433D
:10A620006870C809A8700320694600F0B5F938BD04
:10A6300010B51446012312189B029A4202D9002039
:10A64000C04310BD0B46821E21460920FFF7D4FFF0
:10A65000002010BD10B5054A8905126901430A435F
:10A6600000210820FFF7B9FF002010BD14010020D1
:10A6700038B504466B4601220E212B20FFF788FED9
:10A6800068460078E10640094001C90E014368466A
:10A6900001706B4601220E212B20FFF7ADFF38BD64
:10A6A00010B5002142541C06120A22431B0A491C01
:10A6B0000429F7DB10BD000013B501231A466946D3
:10A6C0000248FDF7A3F900981CBD000030150020DA
:10A6D0007CB5002425466846FFF77FFE04206946C6
:10A6E000220E2D02154322020C5C1443401EF7D5A6
:10A6F000204629467CBD7CB5002425466846FFF7E8
:10A7000074FE04206946220E2D02154322020C5CC1
:10A710001443401EF7D5204629467CBDFCF73CF982
:10A72000FEF72EFDFDF7D2FC3B493C48002522C038
:10A7300005608561C5613A490562C1600838FCF76A
:10A7400065FAFDF7AFFCFDF791FDFDF76DFDFDF737
:10A7500075FC052601223607D1033046FCF707F9C0
:10A76000FEF77EFAFDF76EFBFBF7C4F9FBF792F9F3
:10A770000721B015FFF7E4FC2A4C0A21208A0122A8
:10A780004843A083170339463046FCF7F0F82348C6
:10A79000C82225498830FDF7DBF8244E20790028AF
:10A7A00036D0FEF7EDFC2571FBF7CEFB20700F28AD
:10A7B00009D9012239463046FCF7D9F8FEF756FD93
:10A7C0000022394609E0012251033046FCF7CFF858
:10A7D000FEF74CFD0022012149033046FCF7C7F883
:10A7E000FDF77EFAA08B002801D0401EA083104800
:10A7F000A18B00780843D1D10121C9023046FCF772
:10A80000ADF80028CAD101210846FCF7F1FAC5E7E6
:10A81000FDF766FAC2E70000007C0040A8140020A3
:10A82000FFFF0000C4000020780C0020000400504E
:10A830003600002010B586B01748FCF76CF91421DB
:10A840006846FAF7B4FC15480090032001900020F8
:10A850000290052069460007FBF7C4FF69461048CF
:10A86000FBF7C0FF69460F48FBF7BCFF0121084614
:10A87000FCF7BEFAFF2401342046FCF791FA0A499E
:10A8800008680422104308602046FCF799FAFCF798
:10A890009FFA06B010BD0000A8140020FFFF0000C2
:10A8A00000040050000800500070004010B5012264
:10A8B000920218491848FBF7A5F91648174902886B
:10A8C0008A4225D001807D21C90081804910C18044
:10A8D0000A21018100211E224181D243828101226D
:10A8E000C2810184018241828182C182018381838C
:10A8F0001E23C38602230387782343878287C28768
:10A9000002464032118451849184C18300F02EF8B4
:10A9100010BD0000400D002000FC0008AA550000FA
:10A92000F0B58C4600251026052109078E620E4CD5
:10A9300008E067467F5DE760A768FF07FCD0E7682F
:10A940001F706D1C8542F4DB0020074606E0E760BF
:10A95000A568ED07FCD0E5681D54401C9042F6D375
:10A960008E610020F0BD00000030014070B572B66D
:10A970000124074DA40221462846FBF729F90028A7
:10A9800004D0224603492846FBF7C6F962B670BDDB
:10A9900000FC0008400D0020F0B50025102605271A
:10A9A0009C463F070B46BE620C4C06E0595DE160D9
:10A9B000A168C907FCD0E1686D1C8542F6DB002068
:10A9C00007E06146095CE160A168C907FCD0E16865
:10A9D000401C9042F5D3BE610020F0BD0030014024
:10A9E0000000010203040005405C0000A05C0400BC
:10A9F000C06C0800805C0400E03F1E00E07D1E008B
:10AA000007A9022570889B880A001600010006002D
:10AA10000100020087008D002D001A3152001A3308
:10AA20009A001A351D011A376B003B31BE003B33CB
:10AA30005E013B3596023B37000099599959EB511D
:10AA40008F421E45142E0080EB51F5283333E13A36
:10AA5000703DE13AC235852BC2353333C235C2353C
:10AA6000AE47E13A5138A3305138000000000000F1
:10AA700000000102030406070809030406080C107D
:10AA8000182030000000000102030400ACAA0008F6
:10AA90000000002014010000D09A0008C0AB00089C
:10AAA0001401002044190000E09A00080007040087
:10AAB000091E0805400826091040085608054008E8
:10AAC000261D040008BE1D040008BED8BC401008A6
:10AAD000010000000000C84200000000000000006B
:10AAE0000000000000000000000000000000000066
:10AAF0000000000001000000000000000000000055
:10AB0000000000000000000000005C1200000000D7
:10AB10000000000000000000000000000000000035
:10AB20000000000000000000000000000000000025
:10AB30000000000000000000000000000000000015
:10AB40000000000000000000000000000000000005
:10AB500000000000000000000000000002020400ED
:10AB6000090901020081000000000000010000004E
:10AB700000010000000000000000000000000000D4
:10AB800000000000000000000000000000000000C5
:10AB900000000000000000000000000000000000B5
:10ABA00000000000000000000000000000000000A5
:10ABB0000000000000000000000020000000000075
:04000005080050C1DE
:00000001FF
